:1000000061288F00220884002009282084138F088B
:1000100003195C28F03091000E0880389000F03011
:1000200091030319910003198F0303195C28182801
:100030002B2003010C1820088E1F20088E0803199E
:100040000301900F252880060C28262800000F2881
:10005000841780055C280D080C0403198C0A803075
:100060000C1A8D060C198D068C188D060D0D8C0D35
:100070008D0D5C288F018E00FF308E07031C8F07CB
:10008000031C5C2803308D00DF3048203C288D01A4
:10009000E83E8C008D09FC30031C51288C070318A6
:1000A0004E288C0764008D0F4E280C1857288C1C86
:1000B0005B2800005B28080083130313831264008D
:1000C0000800061483160610831286108316861005
:1000D0008312782032303A200610831606108312DD
:1000E0008614831686108312782032303A206128D5
:1000F00024088C0025088D002B200C08A4000D0876
:10010000A5005F302405A6000630A2001030A00034
:0E01100026088E0004300120080063008D28B0
:02400E00F53F7C
:00000001FF
